:1000000012C02CC02BC087C029C028C027C026C062
:1000100025C024C023C02AC021C020C0AEC01EC03D
:100020001DC01CC01BC011241FBECFE5D4E0DEBF25
:10003000CDBF10E0A0E6B0E0EEEBF3E102C005902A
:100040000D92A037B107D9F712E0A0E7B0E001C0E8
:100050001D92AA3DB107E1F702D1AFC9D1CF1092ED
:100060007200109273001092740008951F920F9204
:100070000FB60F9211248F93EF93FF938CB180935F
:100080007500809174008830B8F4E0917200F0E05F
:100090008CB1EE52FD4F8083809174008F5F80930E
:1000A0007400809172008F5F809372008091720063
:1000B000883011F410927200FF91EF918F910F90A0
:1000C0000FBE0F901F90189580917400882311F433
:1000D000E0E016C0E0917300F0E0EE52FD4FE081E9
:1000E00080917400815080937400809173008F5FC1
:1000F0008093730080917300883011F41092730024
:100100008E2F08955D9BFECF8CB908958091750068
:100110001092750008951F920F920FB60F9211243E
:100120002F938F939F93EF93FF93E091D002F091E1
:10013000D102E754FF4F808190E09BBD8ABD809142
:10014000D0029091D10201969093D1028093D00277
:100150008091D0029091D1028050924020F0109274
:10016000D1021092D002FF91EF919F918F912F9128
:100170000F900FBE0F901F9018951F920F920FB601
:100180000F9211248F939F9385B190E09093BA02C0
:100190008093B9029F918F910F900FBE0F901F9087
:1001A00018950F931F93DF93CF9300D0CDB7DEB791
:1001B0008C018FE890E0D4D6C80181D48093CF021F
:1001C000882311F081E044C089EB90E060E072E0A8
:1001D0008E010F5F1F4FA8017CD38093CF0288232D
:1001E00011F083E035C080E889BF20E02223A9F424
:1001F0008091D0029091D1028F3F9105C9F3C0F355
:1002000089EB90E060E071E0A80163D389819A8175
:100210008F3F9105B1F0A8F021E08091D00290913C
:10022000D1028F3F910509F008F789EB91E060E07A
:1002300071E0A8014ED389819A818F3F910509F021
:10024000B8F619BE80E090E08BD68093CF0280E0B4
:100250000F900F90CF91DF911F910F9108951F93F1
:10026000CF93DF9388EE81BB12BA18BA82E087BBC6
:1002700081E88FBD89E08EBD1DBC1CBC1BBC1ABCB7
:100280008BE085BD14BC84E083BD10BC83E389B9D9
:1002900088E98AB986E880BD80EE87B98FEF86B994
:1002A00010BE7894C8ECD0E015E5829B0EC0959AFC
:1002B00084EC99E0FE013197F1F70197D9F780E6D8
:1002C00090E06FDF89B7816089BF829B95988CEB46
:1002D00092E0FE013197F1F70197D9F760E05D9B5D
:1002E000FECF1CB98091D20290E09093BE02809321
:1002F000BD028091D30290E09093BC028093BB0238
:100300001092720010927300109274008091BB02E0
:100310009091BC022091BD023091BE02582F44271B
:10032000420F531F84EF91E0FE013197F1F70197DF
:10033000D9F76F5F653099F6409370005093710064
:100340008091B9029091BA02880F991F880F991F66
:100350009093BA028093B9028091B9029091BA0247
:100360008417950708F496988091B9029091BA0283
:100370004817590708F4969A4833510508F097989A
:100380004733510508F091CF979A84EC99E0FE012C
:100390003197F1F70197D9F787E690E002DF89B747
:1003A000816089BF82CFDF92EF92FF920F931F93FC
:1003B000D82E7A018B0187FF0BC087E740E050E021
:1003C00060E070E0F0DF823008F040C08FE7D822B4
:1003D000C29A8FEF8FB9779BFECF8FB1C2988FEF04
:1003E0008FB9779BFECF8FB1DFB8779BFECF812F80
:1003F0009927AA27BB278FB9779BFECFC801AA27C9
:10040000BB278FB9779BFECFBB27A12F902F8F2DB6
:100410008FB9779BFECFEFB8779BFECF80E4D816DD
:1004200011F485E906C088E4D81611F487E801C004
:1004300081E08FB9779BFECF9AE02FEF2FB9779BA2
:10044000FECF8FB187FF02C09150C1F71F910F916E
:10045000FF90EF90DF900895EF92FF920F931F931C
:10046000CF93DF937C01E9018091760083FD07C083
:1004700039E0440F551F661F771F3A95D1F781E584
:1004800092DF882309F03AC080E49CE93FEF3FB94E
:10049000779BFECF2FB12F3F19F40197C1F72EC0E4
:1004A0002E3F61F5222733272C1B3D0B2E5F3D4F3E
:1004B000201B310B209739F08FEF8FB9779BFECF40
:1004C0009FB12197D1F7E114F10471F09FEF9FB92B
:1004D000779BFECF8FB1F70180830150104021F050
:1004E0000894E11CF11CF3CF8FEF8FB9779BFECFFF
:1004F0009FB121503040C9F790E001C091E0C29A0D
:100500008FEF8FB9779BFECF8FB1892FDF91CF917E
:100510001F910F91FF90EF900895AF92BF92CF92ED
:10052000DF92EF92FF920F931F93DF93CF9300D050
:1005300000D0CDB7DEB7CCD6C29A8AE09FEF9FB984
:10054000779BFECF2FB18150D1F780E440E050E09F
:1005500060E070E028DF813009F074C088E44AEA86
:1005600051E060E070E01FDF813009F045C06E01AE
:100570000894C11CD11C76019FEF9E012B5F3F4F59
:100580009FB9779BFECF8FB1F70181937F01E2176F
:10059000F307B1F78B81813009F054C08C818A3A1E
:1005A00009F050C000E117E2A8ECAA2EB12C07C058
:1005B000C5010197F1F70150104009F443C089EEDD
:1005C00040E050E060E070E4EEDE882389F756C03A
:1005D0009FEF9FB9779BFECF8FB1F60181936F019B
:1005E000EE15FF05B1F7898186FD03C0F4E0FF2E0B
:1005F0002AC0ECE0FE2E27C089EE40E050E060E02B
:1006000070E0D1DE823028F071E4E72EFF24F3940D
:1006100004C069EEE62E52E0F52E00E117E248EC48
:10062000C42ED12C06C0C6010197F1F7015010402D
:1006300049F08E2D40E050E060E070E0B4DE8823A9
:1006400091F726C0FF24F0927600C29A8FEF8FB9FF
:10065000779BFECF8FB180E0FF2009F481E00F90FF
:100660000F900F900F90CF91DF911F910F91FF90FE
:10067000EF90DF90CF90BF90AF9008958AE740E071
:1006800050E060E070E08FDE882309F4A1CFDACF7C
:1006900080E540E052E060E070E085DE882391F67E
:1006A000D2CFCF92DF92EF92FF920F931F93CF930F
:1006B000DF936C01C0917700D0917800FC0111822A
:1006C00010822481358146815781213031054105D1
:1006D000510509F45AC08E819F81A885B9852817D4
:1006E00039074A075B0708F050C02115310541055D
:1006F000510539F48881833021F42E853F8548895E
:100700005989F601208731874287538721153105A2
:100710004105510579F18EEFE82E8FEFF82E8FEF1E
:10072000082F8FEF182FE20EF31E041F151F8E8166
:100730009F81A885B9850297A109B109E816F90634
:100740000A071B0728F020E030E040E050E016C028
:100750002A8130E040E050E0C801B701EDD59B01AF
:10076000AC018A899B89AC89BD89280F391F4A1F32
:100770005B1F04C02E853F8548895989F60124876F
:1007800035874687578780E001C081E0DF91CF91B0
:100790001F910F91FF90EF90DF90CF9008950F93EE
:1007A0001F93DF93CF9300D000D0CDB7DEB78B017E
:1007B0009C01E0917700F09178006230710581052D
:1007C000910508F477C086819781A085B1850817C7
:1007D00019072A073B0708F06DC08081823021F09D
:1007E000833009F067C022C07727632F522F412F33
:1007F00082859385A485B585480F591F6A1F7B1F85
:1008000098013070220F331FCE01019602E010E0F4
:1008100023DE882309F04EC09A8180E0298130E0F0
:10082000822B932B9C0140E050E048C0B901A80105
:10083000A7E07695679557954795AA95D1F7828554
:100840009385A485B585480F591F6A1F7B1F9801A2
:100850002F773070220F331F220F331FCE010196E6
:1008600004E010E0F9DD882329F58C8190E0A0E018
:10087000B0E0582F4427332722278B8190E0A0E057
:10088000B0E0DC0199278827282B392B4A2B5B2BDA
:10089000898190E0A0E0B0E0282B392B4A2B5B2B1C
:1008A0009A8180E0A0E0B0E0282B392B4A2B5B2B0B
:1008B0005F7004C021E030E040E050E0B901CA01BF
:1008C0000F900F900F900F90CF91DF911F910F918C
:1008D00008954F925F926F927F928F929F92AF9204
:1008E000BF92CF92DF92EF92FF920F931F93CF931D
:1008F000DF933C016B014A01C0917700D0917800F1
:10090000FA0111821082209711F486E0C7C0898114
:1009100080FD02C085E0C2C02A8D3B8D4C8D5D8D6F
:100920008E899F89A88DB98D281B390B4A0B5B0BCB
:10093000CB01A0E0B0E0281739074A075B0708F4AD
:1009400069015301412C72E0572EA0C02E893F89C6
:10095000488D598DDA01C9019170A070B07000976F
:10096000A105B10509F05EC0DA01C90169E0B695DB
:10097000A795979587956A95D1F7FA80FA94F8220A
:10098000C9F4211531054105510529F46E8D7F8D7E
:1009900088A199A105C06AA17BA18CA19DA1FFDEC0
:1009A000623071058105910508F476C06AA37BA3C6
:1009B0008CA39DA300917700109178002AA13BA100
:1009C0004CA15DA12250304040405040F80186814A
:1009D0009781A085B1850297A109B1092817390728
:1009E0004A075B0708F058C0628170E080E090E041
:1009F000A3D49B01AC01F80182899389A489B589AC
:100A0000280F391F4A1F5B1F21153105410551056C
:100A100009F442C02F0D311D411D511D2EA33FA3CE
:100A200048A759A72E893F893170C201821B930BB9
:100A300076018C159D0508F47C016114710419F48C
:100A400080E090E001C0C5014EA15FA168A579A535
:100A5000870102DD882301F5C701A0E0B0E02E89FF
:100A60003F89488D598D280F391F4A1F5B1F2E8BD8
:100A70003F8B488F598FAE0CBF1CCE18DF08F40196
:100A8000808191818E0D9F1D91838083C114D1043B
:100A900009F05CCF80E002C0198281E0DF91CF9144
:100AA0001F910F91FF90EF90DF90CF90BF90AF908C
:100AB0009F908F907F906F905F904F9008952F92AE
:100AC0003F924F925F926F927F928F929F92AF92DE
:100AD000BF92CF92DF92EF92FF920F931F93DF931B
:100AE000CF93CDB7DEB7EF970FB6F894DEBF0FBE4A
:100AF000CDBF4C0120907700309078002114310454
:100B000011F496E0B0C1F1011182CE010196988BEB
:100B10008F8703C00894811C911CF401808180326E
:100B2000C9F38F3219F40894811C911C198A1A8A0E
:100B30001B8A1C8AF4018081813248F4CE010D9613
:100B4000B0DD982F1D8E882309F43AC18CC1CE01E7
:100B500088969FAF8EAFAF85B889FD018BE090E09E
:100B600002C020E2219301972FEF8F3F9207C9F730
:100B700038E01DAE20E002C03BE028E0F4018DAD7E
:100B8000E80FF11D90818F5F8DAF9132B0F09F32F1
:100B9000A1F09E3211F0231728F0383071F49E3204
:100BA00059F30BC0892F81568A3108F49052FD0108
:100BB000E20FF11D90832F5FE1CF1B961C921B97D4
:100BC000913218F491E01B969C93CE010D9669DD4D
:100BD000982F882309F0C9C0498D5A8D6B8D7C8D63
:100BE0002D853E852F703070F5E0220F331FFA956A
:100BF000E1F7CE014D9600E210E02EDC882309F0EB
:100C000056C18D8D882309F448C148A543FD12C003
:100C10002F853889D901FE017D968EAD9FADE817ED
:100C2000F90709F43CC190818C91981719F4319619
:100C30001196F3CF0091770010917800AD84BE84B7
:100C40000894A11CB11CA114B10409F426C1298D7A
:100C50003A8D4B8D5C8D211531054105510509F407
:100C60001CC1C5018F709070892B09F07BC02F5F6C
:100C70003F4F4F4F5F4F298F3A8F4B8F5C8F4D897E
:100C80005E896F89788D411551056105710541F4C3
:100C9000F80184819581A816B90608F0FEC062C0EB
:100CA000F801828190E001979501E4E0369527955F
:100CB000EA95E1F782239323892B09F053C0CB01F6
:100CC000BA016DDD9B01AC016230710581059105B2
:100CD00008F4EDC0F80186819781A085B1852817B9
:100CE00039074A075B0708F0D8C02D8B3E8B4F8B26
:100CF000588FC0907700D09078006EEFE62E6FEF9F
:100D0000F62E6FEF062F6FEF162FE20EF31E041F65
:100D1000151FF60186819781A085B1850297A109EB
:100D2000B109E816F9060A071B0728F020E030E0B1
:100D300040E050E013C0F601228130E040E050E096
:100D4000C801B701F9D29B01AC01F60182899389F0
:100D5000A489B589280F391F4A1F5B1F298F3A8F35
:100D60004B8F5C8FBE86AD8637CF833009F07BC05A
:100D7000EF85F8898385882309F497C074C044FF00
:100D800094C0FDAD8F0E911C5AA8442429A930E0CF
:100D90002429352940E050E0A9013327222778ACE7
:100DA00066248FA990E086299729A0E0B0E0282B3F
:100DB000392B4A2B5B2B298B3A8B4B8B5C8BCBCE05
:100DC0008D8D882309F44EC088A584FD4BC03AA9B7
:100DD00020E089A990E0282B392B40E050E0A901C0
:100DE0003327222798AD80E06FA970E0862B972BE0
:100DF000A0E0B0E0282B392B4A2B5B2BF101268F8A
:100E0000378F40A351A32CAD30E040E050E0522F8B
:100E10004427332722278BAD90E0A0E0B0E0DC012F
:100E200099278827282B392B4A2B5B2B89AD90E0FB
:100E3000A0E0B0E0282B392B4A2B5B2B9AAD80E049
:100E4000A0E0B0E0282B392B4A2B5B2B228F338F6D
:100E5000448F558F168A178A108E118E81E08183F8
:100E600090E001C093E0892FEF960FB6F894DEBFB3
:100E70000FBECDBFCF91DF911F910F91FF90EF90EB
:100E8000DF90CF90BF90AF909F908F907F906F90AA
:100E90005F904F903F902F90089593E069CFF901B4
:100EA0008385882309F46BCF8BCF94E0DCCF91E06E
:100EB000DACFCF92DF92EF92FF920F931F93CF93EF
:100EC000DF93EC016A017B012EEF31E002E010E0DC
:100ED000C3DA882311F043E039C0998180E028818A
:100EE00030E0822B932B85559A4A11F042E02EC0B8
:100EF000CE01B701A60126E330E002E010E0ACDA53
:100F0000882359F4998180E0288130E0822B932B4B
:100F10008654914411F440E019C0CE01B701A601F6
:100F200022E530E002E010E097DA882311F041E09A
:100F30000DC040E0998180E0288130E0822B932B26
:100F40008654914409F441E081E04827842FDF91E1
:100F5000CF911F910F91FF90EF90DF90CF90089568
:100F60004F925F926F927F928F929F92AF92BF92B9
:100F7000CF92DF92EF92FF920F931F93DF93CF9365
:100F8000CDB7DEB7A4970FB6F894DEBF0FBECDBFC6
:100F90004C011092780010927700009709F47CC100
:100FA000BCDA80FF02C082E07CC17E010894E11CB3
:100FB000F11CC70140E050E060E070E07ADF813072
:100FC00021F0AA24BB24650138C0C70140E050E0ED
:100FD00060E070E02EEB31E000E110E03DDA8823C4
:100FE00009F05CC18D81882309F45AC18C8590E099
:100FF000A0E0B0E0D82ECC24BB24AA248B8590E0BE
:10100000A0E0B0E0DC0199278827A82AB92ACA2ADB
:10101000DB2A898590E0A0E0B0E0A82AB92ACA2A94
:10102000DB2A9A8580E0A0E0B0E0A82AB92ACA2A83
:10103000DB2AC701B601A5013CDF833009F42EC1CC
:10104000882309F02DC1CE010196B601A5012DE03E
:1010500030E004E210E000DA882309F01FC19B852C
:1010600080E02A8530E0822B932B7C0100E010E0A9
:10107000E114F1040105110519F58B8D90E0A0E054
:10108000B0E0182F0027FF24EE248A8D90E0A0E026
:10109000B0E0DC0199278827E82AF92A0A2B1B2BC4
:1010A000888D90E0A0E0B0E0E82AF92A0A2B1B2BFB
:1010B000998D80E0A0E0B0E0E82AF92A0A2B1B2BEA
:1010C0002C8130E040E050E0C801B70135D12B0160
:1010D0003C019B8180E02A8130E0822B932BA0E0B1
:1010E000B0E0A80EB91ECA1EDB1EF401A286B386AC
:1010F000C486D586898182839E8180E02D81422F9E
:1011000050E0482B592B55834483988580E02F81EC
:1011100030E0822B932B7C0100E010E0E114F1041D
:101120000105110519F58F8990E0A0E0B0E0182FB6
:101130000027FF24EE248E8990E0A0E0B0E0DC01DF
:1011400099278827E82AF92A0A2B1B2B8C8990E0FB
:10115000A0E0B0E0E82AF92A0A2B1B2B9D8980E049
:10116000A0E0B0E0E82AF92A0A2B1B2B9B8180E043
:101170002A8130E0822B932BA0E0B0E0E81AF90A34
:101180000A0B1B0BE418F5080609170984E05695AD
:1011900047958A95E1F7CA01A0E0B0E0E81AF90A9C
:1011A0000A0B1B0BF401228130E040E050E0C80143
:1011B000B701E1D02E5F3F4F4F4F5F4FF4012683C1
:1011C000378340875187273FFFE03F07F0E04F0715
:1011D000F0E05F0708F464C0275F3F4F4040504095
:1011E00010F083E001C082E0F4018083833041F598
:1011F0002BA130E040E050E0522F44273327222734
:101200008AA190E0A0E0B0E0DC0199278827282B94
:10121000392B4A2B5B2B88A190E0A0E0B0E0282B73
:10122000392B4A2B5B2B99A180E0A0E0B0E0282B62
:10123000392B4A2B5B2B26873787408B518B0DC070
:10124000F40182859385A485B585840D951DA61D21
:10125000B71D86879787A08BB18BF4018481958118
:10126000A4E096958795AA95E1F7A0E0B0E02285E5
:10127000338544855585820F931FA41FB51F840DA8
:10128000951DA61DB71D828B938BA48BB58B1182E8
:10129000909278008092770080E003C081E001C0E6
:1012A00087E0A4960FB6F894DEBF0FBECDBFCF91F6
:1012B000DF911F910F91FF90EF90DF90CF90BF9043
:1012C000AF909F908F907F906F905F904F90089518
:1012D00087B38C6287BBBC9888B38C6388BB80E57E
:1012E0008DB981E08EB908958FB9779BFECF0895AF
:1012F0008FEF8FB9779BFECF8FB108958FB9779B12
:10130000FECF8FB10895982FFB0106C080818FB961
:10131000779BFECF319691509923C1F70895982F6E
:10132000FB0107C080818FB9779BFECF8FB181937E
:1013300091509923B9F70895629FD001739FF001EE
:10134000829FE00DF11D649FE00DF11D929FF00D55
:10135000839FF00D749FF00D659FF00D9927729F8C
:10136000B00DE11DF91F639FB00DE11DF91FBD0117
:10137000CF0111240895A1E21A2EAA1BBB1BFD0167
:101380000DC0AA1FBB1FEE1FFF1FA217B307E40764
:10139000F50720F0A21BB30BE40BF50B661F771FBC
:1013A000881F991F1A9469F760957095809590959C
:0E13B0009B01AC01BD01CF010895F894FFCF61
:1013BE006F622E776176007072652E77617600000F
:00000001FF
